:020000040800F2
:1000000000200020E9300008CD2A0008CF2A00088F
:1000100000000000000000000000000000000000E0
:10002000000000000000000000000000D12A0008CD
:100030000000000000000000D32A0008D52A0008B4
:1000400039310008393100083931000839310008E8
:1000500039310008393100083931000839310008D8
:1000600000000000393100083931000800000000AC
:10007000393100083931000839310008000000002A
:10008000DD2A00083931000800000000393100087D
:10009000000000003931000839310008393100080A
:1000A00000000000393100083931000839310008FA
:1000B000ED2A0008000000003931000800000000AF
:1000C000002243088B4274D303098B425FD3030A97
:1000D0008B4244D3030B8B4228D3030C8B420DD3AA
:1000E000FF22090212BA030C8B4202D31212090238
:1000F00065D0030B8B4219D300E0090AC30B8B4276
:1001000001D3CB03C01A5241830B8B4201D38B0323
:10011000C01A5241430B8B4201D34B03C01A5241C8
:10012000030B8B4201D30B03C01A5241C30A8B420B
:1001300001D3CB02C01A5241830A8B4201D38B02F6
:10014000C01A5241430A8B4201D34B02C01A52419A
:10015000030A8B4201D30B02C01A5241CDD2C3090C
:100160008B4201D3CB01C01A524183098B4201D388
:100170008B01C01A524143098B4201D34B01C01A73
:10018000524103098B4201D30B01C01A5241C308EB
:100190008B4201D3CB00C01A524183088B4201D35A
:1001A0008B00C01A524143088B4201D34B00C01A46
:1001B0005241411A00D20146524110467047FFE7B2
:1001C00001B5002000F0F0F802BDC0460029F7D0CC
:1001D00076E7704703460B437FD4002243088B42E7
:1001E00074D303098B425FD3030A8B4244D3030BBE
:1001F0008B4228D3030C8B420DD3FF22090212BA83
:10020000030C8B4202D31212090265D0030B8B42FE
:1002100019D300E0090AC30B8B4201D3CB03C01AE8
:100220005241830B8B4201D38B03C01A5241430BC3
:100230008B4201D34B03C01A5241030B8B4201D3B3
:100240000B03C01A5241C30A8B4201D3CB02C01A1E
:100250005241830A8B4201D38B02C01A5241430A96
:100260008B4201D34B02C01A5241030A8B4201D385
:100270000B02C01A5241CDD2C3098B4201D3CB012C
:10028000C01A524183098B4201D38B01C01A5241DB
:1002900043098B4201D34B01C01A524103098B42DF
:1002A00001D30B01C01A5241C3088B4201D3CB00CA
:1002B000C01A524183088B4201D38B00C01A5241AD
:1002C00043088B4201D34B00C01A5241411A00D25D
:1002D00001465241104670475DE0CA0F00D04942C6
:1002E000031000D34042534000229C4603098B4236
:1002F0002DD3030A8B4212D3FC22890112BA030ABE
:100300008B420CD3890192118B4208D3890192113F
:100310008B4204D389013AD0921100E08909C309C4
:100320008B4201D3CB01C01A524183098B4201D3C6
:100330008B01C01A524143098B4201D34B01C01AB1
:10034000524103098B4201D30B01C01A5241C30829
:100350008B4201D3CB00C01A524183088B4201D398
:100360008B00C01A5241D9D243088B4201D34B00B3
:10037000C01A5241411A00D20146634652415B10F5
:10038000104601D34042002B00D5494270476346D6
:100390005B1000D3404201B5002000F005F802BD1B
:1003A0000029F8D016E770477047C0460448054B4F
:1003B00010B5834203D0044B002B00D0984710BDEA
:1003C00034010020340100200000000006480749E5
:1003D000091A8B10C90FC91810B5491003D0044B66
:1003E000002B00D0984710BD3401002034010020BC
:1003F0000000000010B5074C2378002B09D1FFF74F
:10040000D5FF054B002B02D0044800E000BF0123BC
:10041000237010BD3401002000000000E03C000803
:10042000054B10B5002B03D00449054800E000BF80
:10043000FFF7CCFF10BDC0460000000038010020CF
:10044000E03C000870B588B0294B1B689868002311
:100450000222002102F096FF00230093254CE26B5C
:10046000802189020A43E263E26B0A400092009A0B
:100470002148224A0260E122520242608360C36046
:10048000036183610C224261C361036201F004F8DD
:10049000626B01231A436263626B1A400192019AF4
:1004A000626B1A436263626B1A400292029A03AC57
:1004B00004250395022204920593023306930795BF
:1004C000A026F6052100300000F02CF90823039344
:1004D00007952100300000F025F9012200211C20A1
:1004E00000F0D8F81C2000F0D9F808B070BDC04664
:1004F000E4000020001002405001002000440040B1
:1005000000B583B00190FA2304489B00012201A9A1
:1005100001F000F8019803B000BDC0465001002072
:1005200070B51600002405E04D1C0878FFF7E8FFC1
:1005300001342900B442F7DB300070BD70B505000E
:10054000114B1968002901D1012070BD0F4B1C68A7
:10055000FA208000FFF7B4FD01002000FFF7B0FD96
:1005600000F0A6F800280DD1032D01D90120ECE7F9
:10057000013000222900404200F08CF8044B1D603D
:100580000020E2E70120E0E7C0000020D4000020C6
:10059000C400002010B50320FFF7D0FF041E02D0D6
:1005A0000124200010BD02F077FAFAE7034A13682D
:1005B000034909685B1813607047C0469C0100201E
:1005C000C0000020014B18687047C0469C01002005
:1005D00070B50400FFF7F6FF0500631C02D0044B62
:1005E0001B68E418FFF7EEFF401BA042FAD370BD72
:1005F000C000002070B5002813DB8308C0339B00C7
:10060000144C1A59944603221040C000FC321500C5
:1006100085406646AE4389010A40824032431A5102
:1006200070BD0F230340083B9B0806339B000A4A1A
:10063000944663445A68944603221040C000FC323A
:10064000140084406546A54389010A4082402A433C
:100650005A60E5E700E100E000ED00E001388023AA
:100660005B0498420FD2094A50600948036A1B0292
:100670001B0AC02109060B43036200239360073362
:100680001360002070470120FCE7C04610E000E046
:1006900000ED00E010B5FFF7ADFF10BD1F231840BF
:1006A0001E3B8340014A13607047C04600E100E0F2
:1006B00010B5FFF7D3FF10BD10B52123C35C022B8B
:1006C00003D004238363012010BD026813680E2148
:1006D0008B431360026813680D398B431360036802
:1006E0000D4A934214D00D4A93420FD080225200FB
:1006F0000B4B5A6021230122C254013B0022C254F9
:10070000436B002B06D098470020DDE71022EFE76F
:100710000122EDE70020D7E7080002401C0002405C
:1007200000000240F0B5D6464F464646C0B500230D
:1007300069E084683C40A446CC68B44065462C43DC
:100740008460446894434A681209944601226546CD
:100750002A409A4022434260C4683C408A68B240C2
:100760002243C2604A68D2004CD59A08140018345B
:10077000A4004A4EA75903241C40E4000F26A640BB
:10078000B743A026F605B04200D180E0444EB04207
:100790007BD00226A64034003C43404E18329200E3
:1007A00094518022B7584A46D2433E004C46A64355
:1007B0004C68E40302D53E004C462643374C802764
:1007C000E6518426A7593E0016404C68A40302D582
:1007D0003E004C462643314C8427E65127683E00B4
:1007E00016404C68E40202D53E004C4626432B4C92
:1007F0002660666832404C68A40201D54A463243FE
:10080000264C626001330C682200DA4041D001229C
:100810009A4025001540A9461442F3D04C68022C9A
:1008200001D0122C10D1DC080834A4002758072668
:100830001E40B6000F25B540AF43BC460F69B74018
:100840003E0065462E4326500468A4465E000324FD
:10085000A2462700B740B846FF4365464446A54335
:10086000AC464C68554625402C00B44065462C43A8
:1008700004604C68651E012D00D85AE7112C00D188
:1008800057E7122C00D067E753E7012682E70026DE
:1008900080E7E0BCBA46B146A846F0BD0018024069
:1008A0000004005003690B4201D001207047002072
:1008B000FCE70000044B5A68520B07231340034A1D
:1008C0009B0098587047C046001002401C3E00082C
:1008D00010B586B001A9294B0A0013CB13C203CB74
:1008E00003C2274B9B683822110019401A420CD1D1
:1008F000234B5A68520B07231340042B00D81900CE
:10090000890001ABC85806B010BD1D4B9A6838234A
:100910001340082B2AD01A4B9A6838231340102B07
:100920000DD0174B9A6838231340202B22D0144B3C
:100930009A6838231340182B15D00020E3E7104B9A
:10094000DA6801210B001340114211D10C4A5168A1
:10095000490B07220A40042A00D813009B0001AA71
:1009600098584000CFE780200002CCE70548CAE74E
:100970000548C8E780200002C5E7C046F83C0008EB
:100980000010024000366E01006CDC0270B582B0CF
:10099000041E00D151E20368DB071CD5C64A9168EA
:1009A00038230B40D16801220A40102B09D0082BB4
:1009B00009D06368002B4FD0A368002B39D10120E8
:1009C0003CE2002AF3D0BC4B1B689B0303D5636851
:1009D000002B00D134E223689B0700D48AE0B64B99
:1009E0009A68382111400E00DA680123134010295B
:1009F00074D0002E00D0ADE0AF4B1B685B0503D573
:100A00006369002B00D11DE2AB4A53681B0C1B0429
:100A1000A1690B435360FFF7D5FD0500A64B1B688A
:100A20005B055ED4FFF7CEFD401B0228F6D90320FC
:100A300004E2A1490B68A14A13400B600B68A04A6D
:100A400013400D000B60FFF7BDFD2B682B690C22D6
:100A50009343A26813432B6163688022520293423E
:100A60001DD0A022D20293421ED0934B1A68934904
:100A70000A401A601A6892490A401A606368002B9B
:100A80001ED0FFF79FFD05008B4B1B689B03A2D474
:100A9000FFF798FD401BC828F6D90320CEE1864A0F
:100AA00011680B431360E9E7834B19688022D20277
:100AB0000A431A601968802252020A431A60DDE76D
:100AC000FFF780FD05007C4B1B689B0383D5FFF778
:100AD00079FD401BC828F6D90320AFE1002B8BD04D
:100AE00087E7002E26D0774B1868FFF727FD0028F0
:100AF00000D0A9E123681B0766D56F4B9A6838239D
:100B00001340182B58D0E369002B00D1A1E06A4AAA
:100B1000136E01210B431366FFF754FD0500664B6E
:100B20001B6E9B0750D4FFF74DFD401B0228F6D9E2
:100B3000032083E1FFF7CCFE5F4B9A68120A0F2374
:100B40001340614A9B009A581F231340D8405F4BC3
:100B50001860C8E76369002B1BD0574A11688023CF
:100B60005B000B431360FFF72DFD0500524B1B6824
:100B70005B0506D4FFF726FD401B0228F6D90320AB
:100B80005CE14D4A53681B0C1B04A1690B43536085
:100B9000B0E7494A13684E490B401360FFF712FD56
:100BA0000500454B1B685B05A4D5FFF70BFD401BFB
:100BB0000228F6D9032041E13F4B1B6E9B0703D56A
:100BC000E369002B00D141E123685B0700D4C7E053
:100BD000394B9A6838231340202B4DD0364BDB6BB2
:100BE000DB0052D4344BDA6B802149050A43DA63C7
:100BF000DB6B0B400193019B01231E00354B1B68EF
:100C0000DB0545D5E368002B68D1E368012B00D1F3
:100C100085E0052B00D188E0274BDA6D01218A435E
:100C2000DA65DA6D03318A43DA65E368002B00D1B7
:100C300085E0FFF7C7FC05001F4BDB6D9B0700D568
:100C40008CE0FFF7BFFC401B234B9842F4D90320F4
:100C5000F4E0194A136E01218B431366FFF7B2FCCF
:100C60000500154B1B6E9B07AED5FFF7ABFC401B79
:100C70000228F6D90320E1E00F4BDB6D9B076FD50F
:100C8000E368002B6CD10120D8E000231E00B5E7FB
:100C9000104A116880235B000B431360FFF792FC3E
:100CA00005000C4B1B68DB05ACD4FFF78BFC401B2D
:100CB0000228F6D90320C1E000100240FFFFFEFF2A
:100CC000FFFFFBFFC40000205C3E0008D4000020B2
:100CD000FFFEFFFF00700040881300006049CB6DED
:100CE00001229343CB65CB6D033293430D00CB655B
:100CF000FFF768FCEB6D2369C0229202134207D113
:100D00002A69584B1A4080239B0213432B617CE7CE
:100D100053490A695348024013430B6175E7504A2F
:100D2000D36D01210B43D3657FE74D4BDA6D042171
:100D30000A43DA65DA6D03390A43DA6575E7FFF7C6
:100D400041FC0500464BDB6D9B0707D5FFF73AFCDE
:100D5000401B454B9842F5D903206FE0012E22D06D
:100D6000236A002B00D173E03D4A916838220A4083
:100D7000102A57D0022B1CD0394B1A683B490A4025
:100D80001A60DA6801218A43DA60FFF71BFC04006D
:100D9000334B1B689B0143D5FFF714FC001B022853
:100DA000F6D903204AE02E4AD36B31490B40D36376
:100DB000D6E72B4A13682D490B401360FFF702FC5E
:100DC0000500274B1B689B0106D5FFF7FBFB401B6B
:100DD0000228F6D9032031E0636A002B04D1FFF723
:100DE00069FD244B984235D91D4AD36801218B43B4
:100DF000616A0B43D360116880235B040B4313606B
:100E0000FFF7E0FB0400164B1B689B0106D4FFF7BD
:100E1000D9FB001B0228F6D903200FE000200DE0CB
:100E200000200BE0012B17D00D4BDA680123134093
:100E3000626A934212D1002000E0012002B070BD2E
:100E40000120FBE70120F9E70120F7E70120F5E7A2
:100E50000020F3E70120F1E70120EFE70120EDE7B3
:100E600000100240FFFFFCFF88130000FFFFFFFEA1
:100E7000FFFFFFEFFF23F40070B504000D00002812
:100E800000D1ABE0574B1A68012313408B421FD3AC
:100E900023689A070ED55B0705D5534A9168E0236E
:100EA000DB010B439360504A936850490B40A168A3
:100EB0000B4393602368DB0755D56368012B1ED075
:100EC000002B3AD1484A126852051DD401206DE02A
:100ED000444A136801218B432B431360FFF772FBD5
:100EE0000600404B1A6801231340AB42D0D0FFF7F5
:100EF00069FB801B3E4A9042F3D9032056E03A4AF0
:100F00001268920300D46BE037498A680720824355
:100F100013438B60FFF756FB0600334B9B68382268
:100F20001A406368DB009A421DD0FFF74BFB801B21
:100F30002F4B9842F1D9032038E0022B07D0042B25
:100F40000BD0294A126E9207DED401202EE0264AE9
:100F500012689201D8D4012028E0234AD26D92076A
:100F6000D2D4012022E01F4B1A6801231340AB4268
:100F70001DD823685B0706D51B4A93681D490B40A3
:100F8000E1680B439360FFF7A3FC174B9A68120AC2
:100F90000F231340184A9B009A581F231340D84030
:100FA000164B1860164B1868FFF7C8FA70BD0D4A4B
:100FB000136801218B432B431360FFF703FB0600EB
:100FC000084B1A6801231340AB42D2D0FFF7FAFA5C
:100FD000801B074B9842F3D90320E7E70120E5E7A0
:100FE0000120E3E70020024000100240FFF0FFFF75
:100FF00088130000FF8FFFFF5C3E0008D400002034
:10100000C4000020014B18687047C046D40000207F
:1010100010B5FFF7F7FF064B9A68120B0723134032
:10102000044A9B009A581F231340D84010BDC04665
:10103000001002403C3E00080268D36801210B43C7
:10104000D3600268916807230B40062B03D0136816
:1010500001210B43136000207047704770477047B1
:10106000704710B50400026813699B070FD5D36859
:101070009B070CD503235B4213610433037703689A
:101080009B699B0763D0FFF7E9FF00232377226862
:1010900013695B0712D5D3685B070FD505235B4245
:1010A00013610733237723689A69C0239B001A4290
:1010B00053D02000FFF7D2FF002323772268136963
:1010C0001B0710D5D3681B070DD509235B4213619D
:1010D0000D3323772368DB699B0745D02000FFF79A
:1010E000BDFF0023237722681369DB0612D5D3687E
:1010F000DB060FD511235B42136119332377236875
:10110000DA69C0239B001A4235D02000FFF7A6FF02
:101110000023237722681369DB0702D5D368DB0736
:1011200030D4226813691B0602D5D3681B0630D45D
:10113000226813695B0602D5D3685B0630D4226847
:1011400013699B0602D5D3689B0630D410BDFFF708
:1011500084FF2000FFF783FF97E72000FFF77DFF64
:101160002000FFF77CFFA7E72000FFF776FF2000B5
:10117000FFF775FFB5E72000FFF76FFF2000FFF7CF
:101180006EFFC5E702235B421361200001F0D0F936
:10119000C7E781235B421361200000F06CF8C7E7CA
:1011A00041235B4213612000FFF75AFFC7E7212369
:1011B0005B421361200000F05DF8C7E703681A4A3C
:1011C000904202D0194A904203D1702293434A6858
:1011D0001343154A90420BD0144A904208D0144A47
:1011E000904205D0134A904202D0134A904203D154
:1011F000124A1340CA681343802293434A69134337
:1012000003608B68C3620B688362074B984205D00A
:10121000084B984202D0084B984201D10B690363F6
:10122000012343617047C046002C01400004004088
:10123000002000400044014000480140FFFCFFFF47
:1012400070B5041E14D03D23C35C002B0AD03D258D
:1012500002236355210001C9FFF7B0FF0123635545
:10126000002070BD3C330022C25401F017FCEEE7B1
:101270000120F6E7704770470268D36806490B40C3
:10128000D360026853692331FF318B435361462396
:101290002022C2547047C046DFFEFFFF4523C35CD7
:1012A000212B01D002207047826880235B019A4283
:1012B00019D0C26A0368196812785A60C36A013388
:1012C000C362438E013B9BB24386002B09D1026867
:1012D000D36880218B43D3600268D36840390B43C5
:1012E000D3600020DFE70369002BE2D1C36A026804
:1012F00011681B88DB05DB0D5360C36A0233C362D0
:10130000DFE70000036A5B060BD5026853690949F1
:101310000B40416A0B435361426A80235B019A424E
:1013200000D070470268536903490B40816A0B4340
:101330005361F6E7FFEFFFFFFF9FFFFF70B504006B
:101340000268136934490B40C1680B43136182681A
:1013500003691A4343691A430168CB682F48034065
:101360001343CB60E169226853692D4803400B4366
:101370005361226853692B490B40A1690B435361A8
:10138000E26980231B019A4221D0FFF741FE8300CE
:1013900018188300C01861688900FEF791FE0600E6
:1013A0006421FEF78DFE050164213000FEF70EFF7B
:1013B000080132306421FEF783FEF0230340AC467F
:1013C00063440F22024021689B188B6070BDFFF7B9
:1013D0001FFE830018188300C01861684900FEF7DB
:1013E0006FFE06006421FEF76BFE050164213000EC
:1013F000FEF7ECFEC80032306421FEF761FE4300C8
:10140000F82252001340AC466344EA3AFF3A0240E5
:1014100021689B188B60D9E7FFDFFFFFF3E9FFFF2F
:10142000FFF7FFFFFFFCFFFFF0B5C64600B5050064
:101430000C0016009846069F2B681B6823401B1B58
:101440005A425341B3421ED17B1CF5D0002F05D028
:10145000FFF7B8F84346C01AB842EDD92A68D368F6
:101460000B490B40D3602A685369A331FF318B438A
:10147000536120234522AB540132AB542433002264
:10148000EA54032000E0002080BCB846F0BDC0460E
:101490005FFEFFFF7047000010B5041E34D04523E7
:1014A000C35C002B26D045232422E2542268D36853
:1014B00016490B40D3602000FFF740FF236A002B42
:1014C0001ED12268136912490B40136122685369C7
:1014D00008218B4353612268D16880239B010B4311
:1014E000D3600023A36420334522A3540132A354C4
:1014F000002010BD44330022C254FFF7CBFFD2E7D7
:101500002000FFF7FFFEDCE70120F2E7FFDFFFFF2F
:10151000FFF7FFFFF0B5C64600B582B004000D002E
:1015200017001E004523C35C202B5CD100295FD02F
:10153000002A5FD0826880235B019A4217D044233F
:10154000E35C012B58D044230122E2540023A3641E
:1015500045332032E254FFF735F880462786678608
:10156000A26880235B019A4208D0002715E0036936
:10157000002BE4D1CB07E2D5012035E02369002B15
:101580001ED0002709E03B882268DB05DB0D536095
:101590000237628E013A92B26286638E002B12D0BD
:1015A00000964346002280212000FFF73DFF0028DF
:1015B00024D1002DE7D02A7823685A600135E8E766
:1015C0002F000025E9E70096434600224021200035
:1015D000FFF72AFF002813D145232022E254013BC4
:1015E0000022E25400E0022002B080BCB846F0BD08
:1015F0000120F9E70120F7E70220F5E70320F3E7F0
:101600000320F1E710B54623C35C202B25D1002928
:1016100025D0002A25D02433C35C012B23D04423BA
:101620000124A446C4544163028742870022826495
:10163000462121344454C2540268D168BC330B4360
:10164000D3600268536961460B4353610268D368F3
:101650001F310B43D360002000E0022010BD0120A9
:10166000FCE70120FAE70220F8E7704710B50268AE
:10167000D36840218B43D36045232022C254FFF717
:10168000F4FF002010BD000010B54623C35C222BE0
:1016900035D1826880235B019A420DD003685A6875
:1016A000436B591C41631A70438F013B9BB24387C4
:1016B000002B0ED0002010BD0369002BEED1426B31
:1016C00003685B68DB05DB0D1380436B0233436308
:1016D000EAE70168CB6820229343CB600168CB68BE
:1016E000084C2340CB6001684B690334FF34A343AB
:1016F0004B614623C25400F079FF0020DBE7022053
:10170000D9E7C046FFFEFFFF10B5406A00234387BC
:10171000438600F08DFF10BD7047000070B582B0A9
:10172000050003681C68DE685A69210706D1A20615
:101730000DD5B2060BD5FFF7A7FF16E00121080073
:101740001040114213D19022520016420FD1E206EE
:1017500001D5F20666D4230602D5330600D56CE027
:10176000640602D5760600D56BE002B070BDE307D3
:1017700005D5F30503D5AB6C01221343AB646307B6
:1017800005D5002803D0AB6C02221343AB64A3073A
:1017900005D5002803D0AB6C04221343AB642307A8
:1017A00005D5002803D0AB6C08221343AB64AB6CA7
:1017B000002BDAD0A40601D5B60621D42B685A69CD
:1017C00040231340AA6C120701D4002B24D0280018
:1017D000FFF752FD2B685A69520619D55A69402104
:1017E0008A435A612B6C002B0ED0184A5A63286C1E
:1017F000FEF762FF0028B8D0286C436B9847B4E727
:101800002800FFF741FFD9E7280000F011FFACE7FF
:10181000280000F00DFFA8E7280000F009FF0023D2
:10182000AB64A2E7002201921A6801925B680193FF
:10183000019B2800FFF770FF8DE72800FFF72EFDC2
:1018400093E72800FFF712FF8FE7C046091700084B
:10185000414B1B78002B4ED0404B1978C9B2404BFE
:101860001B78DBB29C464A2907D8312908D81829A9
:1018700008D8002902D0012100E00421002308E05B
:101880000321FBE70221F9E7364A0020D054013357
:10189000DBB2032BF8D9344B00201870334BFF22F6
:1018A0001A70334B00221880324B5F301A540830C4
:1018B0001A546346FE2B0BD003291DD00CD80129E6
:1018C00020D0022910D1274B01221A705A700BE048
:1018D000254B02221A700EE0042905D1214B01226A
:1018E0001A705A709A70DA70234B1B78012B0DD046
:1018F0006346012B16D070471A4B01221A705A709A
:101900009A70F1E7174B01221A70EDE70329EFD91E
:10191000002304E0134A0121D1540133DBB2032B2D
:10192000F8D9E8E70029E6D00F4B01221A704B1EC8
:10193000DBB20E4A1370012901D0002308E0094BE5
:1019400001221A70D7E7074A0120D0540133DBB2D5
:101950009942F8D8CFE7C04659020020690200201A
:1019600067020020A8010020A3010020C800002079
:10197000A4010020D80100206802002070B56A4B45
:101980001B78002B70D0694A157801236B401370C7
:10199000012D13D0664B1B78DCB2012B13D0644BA6
:1019A0001B78022B1CD00124624B1B78002B23D107
:1019B000002C5AD0604B1A78D2B220E05F4A1388CC
:1019C00001331380E6E75D4B1888FA218900FEF7A2
:1019D000FDFB89B2FA235B009942E5D30024E3E7DB
:1019E000564B18886421FEF7F1FB89B2312901D8E2
:1019F0000124D9E70024D7E74F4B1A78D2B24D4BD8
:101A00001B78012B33D04C4B5B78DBB2012D36D0E9
:101A1000002B4DD0A023DB051968494A11408022D4
:101A200052020A431A60802252049A61414B1B7889
:101A3000022B47D0404B9B78DBB23E4A1278032AF8
:101A400048D03D4AD478E4B2012D49D0002C60D072
:101A5000A023DB0519683B4A11408022D2030A43C8
:101A60001A60802212059A6170BD2200C7E7002C1F
:101A700003D0314B5B78DBB2C8E72300C6E7002A0E
:101A80000CD0A023DB0519682D4A11408022520298
:101A90000A431A60802252009A61C7E7A023DB053F
:101AA0001A6827490A401A60DA680A40DA60BDE716
:101AB000A023DB051A6822490A401A60DA680A4046
:101AC000DA60B3E7002C03D01B4B9B78DBB2B4E7A2
:101AD0002300B2E7002CB7D0174AD478E4B2B3E7BA
:101AE000002B0CD0A023DB051968164A1140802278
:101AF000D2030A431A60802212019A61B4E7A0233C
:101B0000DB051A680F490A401A60DA680A40DA6091
:101B1000AAE7A023DB051A680A490A401A60DA68B6
:101B20000A40DA60A0E7C04659020020A201002066
:101B3000A3010020C8000020A8010020A00100206F
:101B4000FFFFFCFFFFFF3FFF00280AD1064A137882
:101B50009B000B43DBB20548C056002800D0117033
:101B60007047034AF3E7C046B7010020743D000800
:101B7000B601002030B5002826D0274C24681D6807
:101B8000651BAC461C6000280BDD0B785BB2013393
:101B90005BB20B706346C82B09D84A2B15D80123BA
:101BA00006E00B785BB2013B5BB20B70F2E70423FB
:101BB000087840B25BB2984214DB00230B701388A4
:101BC0001BB2632B03DD002030BD0223F0E701339D
:101BD0001BB21380114B01221A70114B00221A8084
:101BE0000120F1E7087840B25B42984212DC002302
:101BF0000B7013881BB2002B01DC0020E4E7013BD3
:101C00001BB21380054B01221A70054B00221A806B
:101C10000120D9E70020D7E754020020500200201D
:101C20005202002070B5041E15D1A0202021C0054D
:101C3000FEF738FE0500012800D02500A020402135
:101C4000C005FEF72FFE012803D064002543E8B24B
:101C500070BD0400F9E701210848FEF723FE0500E6
:101C6000012800D00025A0208021C005FEF71AFE23
:101C700004000128E9D00024E7E7C0460004005032
:101C800010B5A0204021C005FEF70CFE012849D068
:101C900000231C00A0202021C005FEF703FE012820
:101CA00000D0002023000343D8B2214B1870A0209D
:101CB0008021C005FEF7F6FD012836D000231C0068
:101CC00001211C48FEF7EEFD012800D00020230072
:101CD0000343D8B2184B187008211848FEF7E2FDEC
:101CE000431E9841C0B2164B18708021490011481C
:101CF000FEF7D8FD431E9841C0B2124B18708021E8
:101D0000A0200902C005FEF7CDFD431E9841C0B2D8
:101D10000D4B18700D4A002313700D4A13700D4AB5
:101D2000137010BD02231C00B4E702231C00C7E798
:101D3000B701002000040050B6010020001400503C
:101D4000CB000020CA000020C9000020C6010020EE
:101D5000C5010020C401002010B508215A48FEF733
:101D6000A1FD002826D1594B1B78012B17D0584BC9
:101D70001B78002B3AD0574A138801339BB213804B
:101D80001288554B9A4231D9544B1B78002B2DD1D8
:101D9000524B01221A704F4B00221A8026E04B4B07
:101DA000002119704A4B01221A704A4B19804C4B82
:101DB0001A70DCE7454B1B78002B17D1434B0122EF
:101DC0001A70434B00221A70454B1B78002B06D02B
:101DD000424B1B78002B02D1424B01321A703F4A12
:101DE000002313703E4A13703A4A13808021490041
:101DF0003D48FEF757FD002827D13C4B1B78012BAF
:101E00001CD08021A0200902C005FEF74BFD002850
:101E100034D1374B1B78012B29D08021490032481F
:101E2000FEF740FD00283BD0324B1B78002B04D03E
:101E3000304B00221A70304B1A8010BD2B4B002201
:101E40001A702E4B01321A70DBE7284B1B78002BDF
:101E5000D7D1264B01221A70284B1B78002BD0D0EB
:101E6000264B00221A70264B01321A70C9E7204B0C
:101E700000221A70234B01321A70CEE71C4B1B78DC
:101E8000002BCAD11A4B01221A701E4B1B78002B53
:101E9000C3D01C4B00221A701B4B01321A70BCE7D6
:101EA0008021A0300902C005FEF7FCFC0028BBD150
:101EB000104B1B78002BC0D10E4B01221A700E4B19
:101EC00000221A80B9E7C04600140050CB00002061
:101ED000BE010020BC01002087130000C3010020C8
:101EE000BA010020C601002000040050CA000020F2
:101EF000C9000020C2010020C0010020B90100205B
:101F0000C5010020B8010020C401002010B5002048
:101F1000FFF788FE01000020FFF716FE134B144A5E
:101F20001449FFF727FE002802D0134B01221A7034
:101F30000120FFF777FE01000120FFF705FE0028D2
:101F400009D00E4B1B78002B05D00C4B00221A70C9
:101F50000B4B01321A700B4B0B4A0C49FFF70AFE70
:101F6000002802D00A4B01221A7010BDB0010020D7
:101F700062020020B50100205F0200205C02002008
:101F80005E020020AC01002064020020B4010020A9
:101F90006002002010B5294BC2001800D3588018E9
:101FA00082799446C079C1B254000322A24002282B
:101FB0002BD002290FD8002915D0012924D1196866
:101FC00091430A0001210800A04002431A606246C2
:101FD0009140996118E0032924D015D30439C9B27E
:101FE0000129ECD910E06046103001210C0084403A
:101FF0009C61186890431860D8689043D8605A690B
:10200000604681408A435A6110BD196891430A00B5
:1020100001210800A04002431A606246103291403C
:102020009961F1E7196891430A0001210800A04075
:1020300002431A60624691409961E5E7D8010020A9
:1020400030B59BB011496822684601F0B8FB002109
:102050000AE052080133DBB2012AFAD80C4AE40044
:10206000121993710131C9B20C290DD80C006A46BE
:10207000C8008558064BC550121892881B189A80C4
:102080000020D8710023E7E71BB030BD0C3D0008ED
:10209000D80100200C2806D8052900D90521024BBB
:1020A000C0001B18D9717047D801002010B500245A
:1020B00004E02000FFF76EFF0134E4B20C2CF8D9E5
:1020C00010BD000010B55B4A136801331360042B88
:1020D00019D9130000221A60002301E00133DBB29A
:1020E0000C2B10D8544AD9005218D279032AF5D1B2
:1020F000514A0C0088584169121994790122A24072
:102100004A404261EAE74D4A1368013313604C4A82
:10211000934219D9494B00221A60002301E0013390
:10212000DBB20C2B10D8444AD9005218D279042AB9
:10213000F5D1414A0C00885841691219947901225D
:10214000A2404A404261EAE73E4A13680133136005
:102150003D4A934219D93B4B00221A60002301E00B
:102160000133DBB20C2B10D8334AD9005218D27984
:10217000052AF5D1304A0C00885841691219947922
:102180000122A2404A404261EAE7304A1378013313
:10219000DBB21370632B18D9130000221A702C4A7B
:1021A00013780133DBB21370002B0ED01300002222
:1021B0001A70284B1B785BB2012B08D0264B1B787A
:1021C000002B10D0244A013B137000231AE0224B4D
:1021D0001B78632B03D8204A01331370F5E71D4B9E
:1021E000FF221A70F1E71B4B01221A70EDE712492A
:1021F000DA008818807910305158012282408A61B3
:102200000133DBB20C2B14D80B4AD9005218D27907
:10221000062AF5D10D4A11780F4A12789142E6D27A
:10222000054AD900501880798958012282408A6174
:10223000E6E710BDD4010020D8010020D001002025
:10224000C3090000CC01002087130000C901002051
:10225000C8010020CC000020C701002070B53A4B17
:102260001B78002B34D0394B188800B2002803DBD0
:10227000642802DD642000E0002009300A21FDF717
:10228000A9FFC5B20A2D00D90A2500240CE00321BC
:10229000FFF700FF06E00221FFF7FCFE02E000214D
:1022A000FFF7F8FE0134E4B2042C11D80420001B1F
:1022B000C0B22A006300591C8D4201D99D42E6D864
:1022C0009A42E8D88A42EAD90121FFF7E3FEE9E71A
:1022D0001F4B1B78002B34D01E4B188800B20028EF
:1022E00003DB642802DD642000E0002009300A21BD
:1022F000FDF770FFC5B20A2D00D90A2500240CE0B5
:102300000321FFF7C7FE06E00221FFF7C3FE02E04C
:102310000021FFF7BFFE0134E4B2042C11D80920DC
:10232000001BC0B22A006300591C8D4201D99D4296
:10233000E6D89A42E8D88A42EAD90121FFF7AAFEF4
:10234000E9E7FFF7B3FE70BD5A02002062020020E9
:102350005B02002064020020284B1B78002B16D063
:10236000274B1A78D1B2274B1B78DBB2002A0FD14A
:10237000254B573201219954A023DB051968234AC4
:102380001140802252000A431A6010229A6170475D
:1023900001290DD01C4B572200219954A023DB05A5
:1023A000802252039A611A6818490A401A60EEE7BF
:1023B000012B14D0164B1B78012B10D0124B572237
:1023C00006219954A023DB051968104A1140802288
:1023D00052000A431A60802252039A61D7E70A4BDF
:1023E000572200219954A023DB05802252039A61D1
:1023F0001A6806490A401A60C9E7C0465802002018
:102400006C0200206B020020D8010020FFFCFFFFBF
:102410006A020020BFF34F8F034B044ADA60BFF318
:102420004F8FC046FDE7C04600ED00E00400FA050E
:10243000F0B589B003AC14220021200001F042F96C
:10244000244B5A6B012632435A635A6B3240019235
:10245000019A596B022211435963596B0A40029247
:10246000029A5A6B20210A435A631B4B0393A027FD
:10247000FF0521003800FEF755F9184B039300259E
:102480006560A66021003800FEF74CF9FE23039337
:102490006560A560124F21003800FEF743F98023E4
:1024A0005B0003936560A56021003800FEF73AF9F0
:1024B00003966560A66021003800FEF733F9082313
:1024C00003936560A66021000648FEF72BF909B06A
:1024D000F0BDC0460010024013190000E08000006B
:1024E000000400500014005010B5FDF7ABFF034985
:1024F00003480122FFF786F810BDC046C002002045
:102500005001002010B5064800F032FF054800F0E9
:102510002FFF054800F02CFF044800F029FF10BDF4
:10252000843D0008B03D0008CC3D0008F03D0008A7
:1025300010B5254B1868013018600A21FDF746FEDA
:10254000002903D1214A136801331360FFF7BAFD54
:102550001D4B18680A21FDF739FE002900D010BD77
:10256000FFF7FAFBFFF7D2FCFFF708FA184B1B78CE
:10257000002B09D0174B1A88174B9A4204D8154ADA
:10258000138801339BB21380144B1B78002B0CD0A3
:10259000134A138801339BB21380C72BDFD90F4B2B
:1025A00000221A700E4B1A80D9E70E4B1B78002BB5
:1025B000D5D00B4B1A880C4B9A42D0D8084A1388B6
:1025C00001339BB21380CAE740020020540200206E
:1025D000C2010020C0010020032900005002002099
:1025E000520200205D0200202F75000030B583B03C
:1025F000040002680B4B9A4201D003B030BD0A4D73
:10260000287800F09FFB0023019323681A68019249
:102610005B680193019B054801222900FEF7F2FF48
:10262000EBE7C04600440040C002002050010020FB
:1026300000B585B00368124A934201D005B000BDD1
:102640000022009219680091596800910099019246
:1026500019680191596801910199029219680291D2
:1026600059680291029903921A6803925B68039376
:10267000039B044904480122FEF7C4FFDEE7C0467D
:1026800000440040C002002050010020FEE700008E
:1026900010B58EB004AC28220021200001F012F801
:1026A00010220021684601F00DF80F230493F13346
:1026B0000993114B1B68DB04DB0C802212021343CD
:1026C0000A9302230C932000FEF760F900280ED134
:1026D000684607230093053B01930023029303936D
:1026E0000121FEF7C9FB002803D10EB010BDFFF792
:1026F000CDFFFFF7CBFFC046100FFF1F10B50C48F2
:102700000C4B03600C4BC360002343600361836088
:1027100043618361FEF794FD002805D10448FEF76C
:102720008BFC002802D110BDFFF7B0FFFFF7AEFF12
:102730007002002000040040BF12000010B584B0F9
:10274000FDF728FFFFF7A4FFFFF772FEFFF7CCFEAF
:10275000FFF776FCFFF794FAFFF7D0FF002405E0BF
:1027600001212000FFF796FC0134E4B20C2C06D8BE
:102770000A2CF5D003212000FFF78CFCF4E7FFF7CB
:1027800095FC002413E0AA4B1B78002B1ED100F00F
:10279000D1FBC820FDF71CFF00F0C8FA002804D0C8
:1027A00000F0CEFA00F05CFCF6E70134E4B2022C53
:1027B0000CD8FA208000FDF70BFF00F0B7FA0028D4
:1027C000E1D000F0BDFA00F04BFCF6E7FFF79AFE0F
:1027D00083E000F0B5FA00F043FC00F0A7FA00280F
:1027E000F7D1944B1B78002B10D0934B00229A5EAC
:1027F000924B1B881BB29A4200D0A3E0904B1B68FF
:10280000904A12689B1A312B00D9A2E08E4B1B789C
:10281000002B10D08D4B00229A5E8D4B1B881BB273
:102820009A4200D0A2E0864B1B688A4A12689B1A23
:10283000312B00D9A1E0884B1B78002B00D0A9E0F8
:10284000864B1B78002B17D0844B00221A70844BC8
:102850001B78012B00D1A4E0814B01221A70804B20
:102860001878C0B200F036FBFFF776FD7D4B0122F1
:102870001A707D4B00221A807C4B1B78012B00D1F3
:1028800092E07B4B1B78002B00D099E0794B1B78B2
:10289000002B0ED0774B00221A70774B1B78DCB2DE
:1028A000002B00D19BE06F4B01221A706E4B00226F
:1028B0001A80724B1B78002B05D0714B1A88714B14
:1028C0009A4200D99DE05A4B1B78002B05D0664BED
:1028D0001A886D4B9A4200D9A4E0594B1B686B4A89
:1028E00012689B1AC72B00D877E7554B1A68674BBD
:1028F0001A60674B46229B5C222B00D16DE70022B9
:102900000092634803681968009159680091009922
:10291000019219680191596801910199029219680F
:10292000029159680291029903921A6803925B68B6
:102930000393039B46232022C25456491F3AFEF7B5
:1029400061FE4AE73D4B1A883B4B1A80FFF786FC35
:1029500054E7384B00221A70394B1A68394B1A6009
:10296000364B1888C0B200F0BBFA4FE7384B1A88D4
:10297000364B1A80FFF772FC55E7334B00221A7072
:102980002F4B1A68334B1A60314B1888C0B200F0D5
:10299000B0FA50E7304B00221A70012000F0B2FA72
:1029A0004EE72F4B1A705AE7304B02221A7000F094
:1029B000AFFA2C4B01221A702B4B00221A8060E7D1
:1029C0002B4B00241C70224B1C80FFF747FC00F0AF
:1029D000ABFA244B01221A70234B1C8056E7264B7E
:1029E00001321A70002000F08DFA05E0002120006D
:1029F000FFF750FB0134E4B2092CF7D9FFF756FB7F
:102A000051E71E4B002119701D4B00221980184BF5
:102A10001A70184B1A7000F081FA6420FDF7D8FD87
:102A2000FFF7F8FC104B00221A8000F083FA54E7FD
:102A30005D02002060020020D0000020640200201F
:102A400054020020480200205F020020CE00002037
:102A500062020020440200205E020020C601002025
:102A60006C0200205002002052020020C30100200E
:102A7000C5010020C40100205C020020C20100202A
:102A8000C0010020032900002F7500004C02002027
:102A900050010020C00200207047000000B583B044
:102AA000094AD16B02231943D163D26B13400193BE
:102AB000019B002201211020FDF7ECFD1020FDF705
:102AC000EDFD03B000BDC046001002407047FEE7B8
:102AD0007047704710B5FDF769FD10BD10B502488D
:102AE000FEF7BFFA10BDC0467002002010B50248C4
:102AF000FEF714FE10BDC046500100200D494B6882
:102B00001B0C1B040C4A1268D204D20C1343802203
:102B1000920113434B604B68084A1340084A1268FD
:102B200012040848024013434B60074B80221205F1
:102B30009A60704700100240040FFF1FFFFF00FE65
:102B4000A40FFF1F0000FF0100ED00E010B50023FF
:102B500008E09A008021090551180868064950507C
:102B60000133DBB22F2BF4D9044B802292059A60FB
:102B7000FFF7E4FD002010BD0000002000ED00E0A4
:102B80000022094B1B681B060AD40132074B9A42EC
:102B900008D8054B1B681B07F3D5034B5B68F0E7B0
:102BA000014B58607047C04600440040A0860100B9
:102BB00070B5022444404C40E4B254400F4B5525BC
:102BC0001D7055355D7098700220D87019715A715A
:102BD0009C71002405E0094B185DFFF7D1FF01341B
:102BE000E4B2062CF7D90022054B1B685B0603D420
:102BF0000132044B9A42F7D970BDC046B80200209A
:102C000000440040A086010010B50A000100022027
:102C1000FFF7CEFF10BD000010B50C00344B1B7841
:102C2000002B02D1324B01221A70002225E0032929
:102C30003AD009D8012919D002291CD12D490B708D
:102C40002D4B0121197016E0042914D12B490B706A
:102C500011E00D290FD12A490978002902D11BB2B0
:102C600028490B80284B0121197004E027490B707B
:102C7000214B012119700132D2B2A24231D253004C
:102C8000DBB2C15C0133C35C09291ED0CFD90C294A
:102C900010D0DED80A291ED00B29ECD11C490B70AC
:102CA0001C4B01211970E6E71B490B70124B0121E7
:102CB0001970E0E712490978002902D11BB21749BF
:102CC0000B80174B01211970D5E716490B70114B7A
:102CD00001211970CFE714490B700E4B01211970B7
:102CE000C9E7FFF7BBFAFFF737FBFEF7B1FD10BDF1
:102CF0005D0200206B0200205802002066020020C6
:102D000050020020620200205A0200206C020020C3
:102D100067020020590200206A020020640200209D
:102D20005B0200206902002068020020034B1B7830
:102D3000D8B2002B00D001207047C046C10200204D
:102D40007047000030B55B4B1B785B015A4A9B18FB
:102D50005A4A1278002A0ED059490A88013292B292
:102D60000A80FA2189008A4208D9544A0021117048
:102D7000534A118002E0524A002111804F4A1278D2
:102D8000002A08D0012A2DD0022A38D0032A42D0A6
:102D9000042A55D030BD55280CD0A028FAD1A02245
:102DA0001A70484B1B78DBB2012B0AD9464B002224
:102DB0001A70EFE71870444B01321A703F4B1A70CB
:102DC000E8E73C4A1378DBB240499F38C85413788F
:102DD000013301210B4013703A4A13780133DBB2FF
:102DE0001370E3E7AA2803D0344B00221A70D1E70E
:102DF0005870354B01321A70304B1A70CAE7324A9C
:102E0000944611784A1CD2B26446227058542B4B17
:102E100003221A70BEE72C4A944611784A1CD2B29B
:102E20006446227058540530C0B2294B1870234BA9
:102E300004221A702028ADD900221A702270A9E746
:102E4000214A11788C460131C9B21170614658543B
:102E500011781F4A127891429CD39978DA7815003C
:102E60005140002204E0141D1C5D61400132D2B2C9
:102E7000AA42F8D3814205D0104B00221A70124B9F
:102E80001A7087E70F4B1B78DBB2012BF4D8094A85
:102E90001378DBB20C490978C9B20C48C1541378D5
:102EA000013301210B401370064A13780133DBB262
:102EB0001370E1E7C3020020CC020020B40200201E
:102EC000B2020020C1020020C4020020C80200207B
:102ED000B002002010B501000120FFF795FE10BDE3
:102EE00010B50100642800D964210C20FFF78CFE86
:102EF00010BD10B50100642800D964210D20FFF732
:102F000083FE10BD10B501000420FFF77DFE10BD4B
:102F100010B500210220FFF777FE10BD10B500218B
:102F20001220FFF771FE10BD10B500211320FFF72E
:102F30006BFE10BD10B5002200210120FFF738FE06
:102F400010BD000010B5374B1B78DCB2002B02D14E
:102F5000344B01221A70092844D00ED90C2851D0C4
:102F60001FD80A2846D00B2831D12F4B19702F4B70
:102F700001221A70FEF76CFC29E003282AD00BD836
:102F800001281DD0022822D1294B1970294B01227A
:102F90001A70FFF7E1F91AE0042818D1264B1970CE
:102FA00015E00D2813D1254B1B78002B02D109B257
:102FB000234B1980234B01221A70FFF74FF906E0CB
:102FC000214B19701B4B01221A70FFF7C5F9002C19
:102FD00025D010BD1D4B1970164B01221A70FFF73A
:102FE000BBF9F4E71A4B1970104B01221A70FEF767
:102FF0002FFCECE7174B19700C4B01221A70FEF7EF
:1030000027FCE4E70D4B1B78002B02D109B2124BD1
:103010001980124B01221A70FFF720F9D7E7FFF74A
:1030200089FFD6E75D0200206702002059020020D8
:103030006B0200205802002066020020500200208F
:10304000620200205A0200206C0200206A02002066
:103050006902002068020020640200205B02002058
:1030600010B51D4B1B78002B20D01C4B187840014D
:103070001B4A80181B78DBB21A4AD35CDBB2062BE2
:1030800007D98378C278812B11D0013BDBB2012BA9
:103090001AD9124A1378013301210B40137072B60A
:1030A0000D4A1378013BDBB2137062B610BD022AE1
:1030B00005D0EED901790530FFF7AEFDE9E741799A
:1030C0000079FFF73FFFE4E7022AE2D14179007976
:1030D000FFF738FFDDE7C046C1020020C202002032
:1030E000CC020020C80200200D488546FFF706FDEF
:1030F0000C480D490D4A002302E0D458C450043353
:10310000C4188C42F9D30A4A0A4C002301E0136028
:103110000432A242FBD300F02BFBFFF717FDFEE7C2
:1031200000200020C000002034010020643F00087F
:10313000340100205C040020FEE70000002310B5ED
:10314000040003604360836081814366C281036140
:1031500043618361190008225C3000F0B3FA0B4B25
:10316000246263620A4BA3620A4BE3620A4B236345
:103170000A4B9C4205D00A4B9C4202D0094B9C4210
:1031800003D12000583000F017FB10BDF1340008C7
:1031900019350008513500087D3500080C03002062
:1031A00074030020DC03002010B5034A03490448DF
:1031B00000F06CF810BDC046D8000020E93A0008C5
:1031C000E800002041680B4B10B50400994201D083
:1031D00000F08AFCA168084B994202D0200000F060
:1031E00083FCE168054B994202D0200000F07CFC92
:1031F00010BDC0460C03002074030020DC03002037
:1032000010B5094B094A04211A6009480022FFF74A
:1032100095FF012209210748FFF790FF02221221A2
:103220000548FFF78BFF10BD44040020A9310008BA
:103230000C03002074030020DC03002010B50248BA
:1032400000F0BBFA10BDC0464D04002010B5024886
:1032500000F0B4FA10BDC0464D04002010B50400C3
:10326000FFF7ECFF236A002B02D0FFF7EFFF10BD42
:10327000044B2362044B1B68002BF6D1FFF7C0FF01
:10328000F3E7C046C531000844040020F7B5140038
:10329000002600900191A5686768013F04D5246865
:1032A000002CF8D13000FEBDAB89012B08D90E22CD
:1032B000AB5E013304D029000098019B9847064378
:1032C0006835EAE7036A70B505000E008468002BD4
:1032D00001D1FFF7C3FF636EDB0705D4A3899B050C
:1032E00002D4A06D00F069FAA3891B0702D52369F7
:1032F000002B1ED12100280000F088F9002818D0EA
:1033000001256D42636EDB0705D4A3899B0502D4BA
:10331000A06D00F053FA280070BD002B04DAA269FA
:10332000934217DB0A2915D023685A1C22601970B2
:103330000136A3683178013BA3600029EDD18B42AF
:103340000FDA220028000A3100F01EF90130D7D030
:103350000A25D7E72200280000F016F90130E7D14E
:10336000CEE723685A1C22600A221A70F0E7000098
:1033700010B5034B01001868FFF7A4FF10BDC0464D
:10338000E4000020F0B51D00574B85B01E68040016
:103390000F000092002E05D0336A002B02D13000BE
:1033A000FFF75CFF009B022B05D0012B00D997E0B3
:1033B000002D00DA94E0636EDB0705D4A3899B053A
:1033C00002D4A06D00F0F9F92100300000F08CFB70
:1033D000616B002908D023004433994202D03000A9
:1033E00000F0F6F9002363630023A3616360A389FF
:1033F0001B0603D53000216900F0EAF9A3893B4A96
:103400001340A381009B022B60D003AB210030004E
:1034100002AA00F095FBA3891843A081002D24D1B6
:10342000029D280000F01EFA0195071E48D1029B5C
:103430000193AB423FD101256D420C22A35E0222D3
:103440001A43A2810022A260220047322260226138
:103450000122616E6261114204D19B0502D4A06D0C
:1034600000F0ACF9280005B0F0BD002FD9D0336AC8
:10347000002B02D13000FFF7F1FE009B012B03D19E
:10348000A389009A1A43A2810C22A35E0822190084
:10349000276027616561114013421BD0DA0717D5F9
:1034A00000226D42A260A561626ED20701D49B0525
:1034B00012D50025D6E7019800F0D4F9071EBAD03E
:1034C0008023A289019D1343A381D0E70025B4E79F
:1034D000A560E9E7A160E7E7A06D00F06FF9E8E714
:1034E00001256D42BEE7C046E40000205CF3FFFF0B
:1034F00070B50C000E25495F00F012F9002803DBBF
:10350000636D1B18636570BDA389024A1340A381D4
:10351000F9E7C046FFEFFFFFF8B51F008B890500F4
:103520000C001600DB0505D50E23C95E0022022320
:1035300000F0E2F8A389054A28001340A381320075
:103540000E23E15E3B0000F0FFF8F8BDFFEFFFFF48
:1035500070B50C000E25495F00F0CEF80C22A35E7A
:10356000421C03D1044A1340A38170BD8022520142
:103570001343A3816065F8E7FFEFFFFF10B50E234B
:10358000C95E00F0A7F810BDF8B505000F001400E3
:10359000002804D0036A002B01D1FFF75FFEA36966
:1035A000A360A3891B0702D52369002B09D1210041
:1035B000280000F02BF8002803D0012676423000C6
:1035C000F8BD23692068C01A6369834205DC2100C5
:1035D000280000F089FA0028EFD1A3680130013BF0
:1035E000A3602368FEB25A1C22601F706369834285
:1035F00004D0A389DB07E2D50A2EE0D12100280000
:1036000000F072FA0028DAD0D7E700002C4B70B532
:10361000050018680C00002804D0036A002B01D1B3
:10362000FFF71CFE0C22A35E1A0721D4DA0607D48A
:1036300009222A60402201201343A381404238E03E
:103640005A0712D5616B002908D0230044339942F0
:1036500002D0280000F0BCF8002363632422A38971
:103660009343002262602269226008221343A381EF
:103670002369002B0BD1A0238022A1899B009200FB
:103680000B40934203D02100280000F083FA0C2263
:10369000A35E01211A000A400B420BD00022A26057
:1036A00062695242A26100202269824201D11A0657
:1036B000C0D470BD990700D46269A260F3E7C04628
:1036C000E400002003008218934200D17047197073
:1036D0000133F9E7002370B5064C050008002360AC
:1036E00000F0C8FA431C03D12368002B00D02B60E4
:1036F00070BDC0464804002070B5050008001100E8
:103700000022064C22601A0000F0CCFA431C03D1C0
:103710002368002B00D02B6070BDC04648040020F9
:1037200070B50500080011000022064C22601A0046
:1037300000F0C0FA431C03D12368002B00D02B609B
:1037400070BDC0464804002070B505000800110097
:103750000022064C22601A00FCF7E2FE431C03D153
:103760002368002B00D02B6070BDC04648040020A9
:1037700070B500260C4C0D4D641BA410A64209D157
:10378000002600F0ADFA0A4C0A4D641BA410A642B4
:1037900005D170BDB300EB5898470136EEE7B30092
:1037A000EB5898470136F2E79C3E00089C3E000823
:1037B000A03E00089C3E00087047704770470023F9
:1037C00010B59A4200D110BDCC5CC4540133F8E767
:1037D00070B50500002910D00C1F2368002B00DAFB
:1037E000E418280000F0EAF81D4A1368002B05D100
:1037F00063601460280000F0E9F870BDA34208D9A6
:10380000206821188B42F3D119685B680918216080
:10381000EEE71A005B68002B01D0A342F9D91168CA
:103820005018A0420BD1206809185018116083422B
:10383000E0D118685B68411811605360DAE7A04274
:1038400002D90C232B60D5E7206821188B4203D1C5
:1038500019685B680918216063605460CAE7C04654
:103860005404002010B5034B0100186800F026F83E
:1038700010BDC046E400002070B50F4C0E0021685A
:103880000500002902D100F0E3F920603100280092
:1038900000F0DEF9431C03D101246442200070BD16
:1038A0000323C41C9C43A042F8D0211A280000F036
:1038B000CFF90130F2D1EFE750040020F7B5032231
:1038C000CB1C9343083305001F000C2B34D20C276C
:1038D000B94233D8280000F071F8374E33681C0025
:1038E000002C2FD139002800FFF7C6FF0400431C2D
:1038F0005FD134680094009B002B4AD19C4252D087
:1039000023682800E3180099019300F0A1F9019BB6
:10391000834248D123682800FF1A3900FFF7ACFF23
:10392000013040D02368DB19236033685A68002ACD
:1039300033D1009B336019E0002BC9DA0C232B60D4
:103940000020FEBD2168C91B20D40B290AD9E21929
:103950002760A34204D1326063681160536005E0C0
:103960005A60F9E76268A3420ED13260280000F085
:103970002DF8200007220B30231D9043C21A9842D5
:10398000DFD01B1AA350DCE75A60EFE7230064681E
:10399000A6E7009C63680093ADE71A005B68A3424A
:1039A000FBD10023DAE70C2328002B6000F00EF88F
:1039B000C6E70760DAE7C0465404002010B50248A5
:1039C000FFF7FBFE10BDC0464C04002010B50248B6
:1039D000FFF7F4FE10BDC0464C040020F7B50C22E2
:1039E0008B5E05000C001A0757D44A68002A02DCD7
:1039F0000A6C002A4FDDE76A002F4CD0002280219C
:103A00002E682A601A0049010A400B4234D0626DC8
:103A1000A3895B0706D56368D21A636B002B01D0BC
:103A2000236CD21A00232800E76A216AB8470C23C6
:103A3000E25E431C06D129681D2947D8294BCB409B
:103A4000DB0743D50023636023692360D20405D5D7
:103A5000431C02D12B68002B00D16065616B2E6086
:103A6000002918D023004433994202D02800FFF7E0
:103A7000AFFE002363630EE001232800216AB847EC
:103A80000200431CC4D12B68002BC1D01D2B01D0D8
:103A9000162B1AD12E6000201DE00E69002EFAD0E0
:103AA0000F680E60BA1B019200229B0700D14A6981
:103AB000A260019B002BEEDDA36A32001F002800EC
:103AC000019B216AB847002806DCA2894023012017
:103AD0001343A3814042FEBD019B36181B1A01937C
:103AE000E7E7C046010040200B6970B505000C00F7
:103AF000002B02D11D00280070BD002804D0036AED
:103B0000002B01D1FFF7AAFB0C22A35E002BF1D002
:103B1000626ED20704D49B0502D4A06DFFF74DFE60
:103B200028002100FFF75AFF636E0500DB07E2D48F
:103B3000A3899B05DFD4A06DFFF740FEDBE7000003
:103B400070B50E001D000E23C95E140096B000294A
:103B50000CDA80210B00B2891340114214D180226B
:103B6000D20000202B60226016B070BD6A4600F0C3
:103B70004BF80028EDDBF022019B12021340044AAF
:103B80009B185A425341EAE700234022E9E7C04626
:103B900000E0FFFFF7B502258B8906000C001D42EF
:103BA00006D0230047332360236101236361F7BDFF
:103BB0006A4601ABFFF7C4FF009F30003900FFF7F2
:103BC0007DFE0C22A35E002806D19A05EFD40322C5
:103BD00093431D43A581E4E780221343A381019B06
:103BE000206020616761002BE1D030000E23E15E90
:103BF00000F01CF80028DAD00323A2899A43023B84
:103C00001343A381D3E70000002370B5064C0500E1
:103C100008001100236000F035F8431C03D123682D
:103C2000002B00D02B6070BD48040020002370B52D
:103C3000064C05000800236000F02CF8431C03D15B
:103C40002368002B00D02B6070BDC04648040020C4
:103C5000002370B5064C05000800236000F032F820
:103C6000431C03D12368002B00D02B6070BDC046DD
:103C70004804002058220120014B40421A6070473E
:103C80004804002058220120014B40421A6070472E
:103C9000480400205822024B00201A607047C0469A
:103CA0004804002058220120014B40421A6070470E
:103CB0004804002058220120014B40421A607047FE
:103CC00048040020044A1368002B03D01818106021
:103CD00018007047014BF9E75804002060040020E9
:103CE000F8B5C046F8BC08BC9E467047F8B5C0465B
:083CF000F8BC08BC9E467047B9
:103CF80000093D0000127A000024F40040865101BA
:103D080000366E0100000050020000000004005060
:103D18008000000000040050400000000004005033
:103D280020000000000000500100000000040050C6
:103D380004000000000400501000000000040050BF
:103D480008000000000000500010000000040050AF
:103D580002000000000000501000000000000050A9
:103D68000001000000000050000800000001FF00F2
:103D7800FF000001010000FF00FF01000D0A3D3DAA
:103D88003D3D3D3D3D3D3D3D3D3D3D3D3D3D3D3D5B
:103D98003D3D3D3D3D3D3D3D3D3D3D3D3D3D3D3D4B
:103DA8003D3D3D3D3D3D0D002020537065616B65F7
:103DB8007220436F6E74726F6C2050616E656C0D6B
:103DC80000000000202057616974696E6720666FE3
:103DD80072206D61696E626F6172642064617461E2
:103DE8002E2E2E0D000000003D3D3D3D3D3D3D3D4C
:103DF8003D3D3D3D3D3D3D3D3D3D3D3D3D3D3D3DEB
:103E08003D3D3D3D3D3D3D3D3D3D3D3D3D3D3D3DDA
:103E18000D00000000093D0000127A000024F400A3
:103E28004086510100366E0100093D0000093D0041
:103E380000093D0000000000000000000000000034
:103E48000000000001000000020000000300000064
:103E58000400000000000000000000000000000056
:103E6800000000000000000000000000000000004A
:103E78000000000001000000020000000300000034
:103E88000400000006000000070000000800000011
:043E9800090000001D
:043E9C0021040008F5
:043EA000F50300081E
:103EA400000000000000000000000000000000000E
:103EB40000000000000000000000000000000000FE
:103EC40000000000000000000000000000000000EE
:103ED40000000000000000000000000000000000DE
:103EE40000000000000000000000000000000000CE
:103EF40000000000000000000000000000000000BE
:103F040000000000000000000000000000000000AD
:103F1400000000000000000000000000000000009D
:103F2400000000000000000000000000000000008D
:103F3400000000000000000000000000000000007D
:103F4400000000000000000000000000000000006D
:103F5400000000000000000000000000000000005D
:103F64000100000004000000FF0101010100FFFF47
:103F7400FFFF000000127A000000000003000000B0
:103F84000C030020E8000020000000000C030020C7
:103F940074030020DC030020000000000000000087
:103FA400000000000000000000000000000000000D
:103FB40000000000000000000000000000000000FD
:103FC40000000000000000000000000000000000ED
:043FD40000000000E9
:04000005080030E9D6
:00000001FF
